:100000000C9408050C944F050C944F050C944F0567
:100010000C944F050C944F050C944F050C944F0510
:100020000C944F050C944F050C94830C0C944F05C5
:100030000C942D1B0C944F050C944F050C944F05FC
:100040000C944F050C944F050C944F050C944F05E0
:100050000C944F050C94CD1B0C944F050C944F053C
:100060000C944F050C944F050C944F050C944F05C0
:100070000C944F050C944F050C944F050C944F05B0
:100080000C944F050C944F050C944F050C944F05A0
:100090000C944F050C944F050C944F050C944F0590
:1000A0000C944F050C944F050C944F05790D9B0D46
:1000B000890E9B0D890EE00D030E890E580E6B0EF6
:1000C000701170119D119D11F81134122C142C1403
:1000D0004C122C144713471302142C142C1418140C
:1000E0001F141A16041D1B062021150807091905DF
:1000F00022231C170A0B11801E352B39797A7B2C91
:100100002425180C0E0D1080742A31287C7D7E7FEA
:1001100026271213330F36802D2E302F3438378098
:10012000253032583A20253038620A000A722F638F
:100130002030313233343536370A005B735D004B83
:100140006579626F6172642073746172742E0A0043
:1001500055534220636F6E666967757265642E0A37
:10016000005B575D005B535D005B525D005B445D6F
:10017000005B435D001203480048004B0042002032
:10018000006D006F00640000000E0374002E006D0F
:10019000002E006B002E0000000403090409028DEC
:1001A00000050100A032090400000103010100095B
:1001B00021110100012240000705810308000A09FE
:1001C0000401000103010200092111010001224D77
:1001D000000705820308000A090402000103000069
:1001E00000092111010001223600070583030800E0
:1001F0000A090403000203000000092111010001A3
:1002000022220007058403200001070504032000C3
:10021000010904040001030000000921110100018B
:10022000223900070585032000011201100100009A
:100230000008EDFEFECA04010102000105010906E5
:10024000A101050719E029E71500250195087501A9
:10025000810205081901290595057501910295018D
:10026000750391010507190029F71500250195F877
:1002700075018102C00631FF0974A10109751500DD
:1002800026FF009520750881020976150026FF00DB
:10029000952075089102C005010980A1018502160B
:1002A000810026B7001A81002AB7007510950181D8
:1002B00000C0050C0901A1018503160100269C025E
:1002C0001A01002A9C02751095018100C0050109E0
:1002D00002A1010901A1000509190129051500253F
:1002E00001950575018102950175038101050109DB
:1002F0003009311581257F95027508810609381569
:1003000081257F950175088106050C0A3802158143
:10031000257F950175088106C0C005010906A10168
:10032000050719E029E715002501950875018102E7
:1003300095017508810105081901290595057501C3
:1003400091029501750391010507190029FF150018
:1003500026FF00950675088100C00A002530325836
:1003600020006B6579626F6172645F7265706F7295
:10037000743A20004C45443A20253032580A006433
:10038000656C5F6B65795F6269743A2063616E27A3
:10039000742064656C3A20253032580A0061646428
:1003A0005F6B65795F6269743A2063616E277420C0
:1003B0006164643A20253032580A004F6E657368D4
:1003C0006F743A2074696D656F75740A00290A00AC
:1003D0002575002F002575005D280025640020008C
:1003E000256400200025640020002564007C002591
:1003F000303258006D6F7573656B6579205B627480
:100400006E7C782079207620685D287265702F6177
:10041000636C293A205B006D6B5F776865656C5F84
:1004200074696D655F746F5F6D6178203D20256430
:100430000A006D6B5F776865656C5F6D61785F73EF
:1004400070656564203D2025640A006D6B5F7469EA
:100450006D655F746F5F6D6178203D2025640A00D3
:100460006D6B5F6D61785F7370656564203D2025FD
:10047000640A006D6B5F696E74657276616C203D15
:100480002025640A006D6B5F64656C6179203D20F6
:1004900025640A006D6B5F776865656C5F74696DD4
:1004A000655F746F5F6D6178203D2025640A006D83
:1004B0006B5F776865656C5F6D61785F73706565AC
:1004C00064203D2025640A006D6B5F74696D655F73
:1004D000746F5F6D6178203D2025640A006D6B5F4D
:1004E0006D61785F7370656564203D2025640A0046
:1004F0006D6B5F696E74657276616C203D2025645A
:100500000A006D6B5F64656C6179203D2025640A8B
:10051000000A00257500363A20776865656C5F74BF
:10052000696D655F746F5F6D61783A20000A002520
:100530007500353A20776865656C5F6D61785F732B
:10054000706565643A20000A00257500343A20740D
:10055000696D655F746F5F6D61783A20000A0025F0
:100560007500333A206D61785F73706565643A2079
:10057000000A00257500323A20696E746572766152
:100580006C286D73293A20000A00257500313A2045
:1005900064656C6179282A31306D73293A20000A2C
:1005A000092D2056616C756573202D0A004D3E00A3
:1005B0004D25643E20003F007365742064656661CC
:1005C000756C740A00433E2000776865726520648C
:1005D000656C74613A20637572736F723D25642C8B
:1005E00020776865656C3D25640A536565206874ED
:1005F00074703A2F2F656E2E77696B697065646928
:10060000612E6F72672F77696B692F4D6F757365F8
:100610005F6B6579730A000A092D204D6F7573654C
:100620006B6579202D0A4553432F713A097175691D
:10063000740A313A0964656C6179282A31306D7326
:10064000290A323A09696E74657276616C286D7395
:10065000290A333A096D61785F73706565640A34FD
:100660003A0974696D655F746F5F6D61780A353A38
:1006700009776865656C5F6D61785F737065656447
:100680000A363A09776865656C5F74696D655F74F1
:100690006F5F6D61780A0A703A097072696E742032
:1006A00076616C7565730A643A09736574206465D4
:1006B0006661756C74730A75703A092B310A646F40
:1006C000776E3A092D310A706775703A092B31300F
:1006D0000A7067646F776E3A092D31300A0A7370B9
:1006E000656564203D2064656C7461202A206D611D
:1006F000785F7370656564202A2028726570656173
:1007000074202F2074696D655F746F5F6D61782947
:100710000A003F004D3E2000433E20004C25640A65
:10072000000A092D20436F6E736F6C65202D0A45FA
:1007300053432F713A09717569740A6D3A096D6FE7
:100740007573656B65790A000A092D204D6167692B
:1007500063202D0A643A0964656275670A783A096C
:100760006465627567206D61747269780A6B3A0915
:100770006465627567206B6579626F6172640A6D8A
:100780003A096465627567206D6F7573650A763A1C
:100790000976657273696F6E0A733A0973746174CE
:1007A00075730A633A09636F6E736F6C65206D6FC2
:1007B00064650A302D343A096C61796572302D34E4
:1007C000284631302D4634290A506175733A096242
:1007D0006F6F746C6F616465720A6E3A094E4B52AA
:1007E0004F0A003F004E4B524F3A206F66660A0098
:1007F0004E4B524F3A206F6E0A0074696D65725FFE
:1008000072656164333228293A202530346C580AE5
:10081000006B6579626F6172645F6E6B726F3A2014
:1008200025580A006B6579626F6172645F69646C58
:10083000653A2025580A006B6579626F6172645FC2
:1008400070726F746F636F6C3A2025580A00686F7E
:1008500073745F6B6579626F6172645F6C656473FA
:1008600028293A2025580A000A092D20537461745A
:100870007573202D0A004743433A20342E392E3217
:10088000204156522D4C4942433A20312E382E30C9
:1008900073766E204156525F415243483A2061764A
:1008A00072350A004F5054494F4E533A204C55462A
:1008B00041204D4F5553454B4559204558545241C1
:1008C0004B455920434F4E534F4C4520434F4D4DC0
:1008D000414E44204E4B524F204B45594D41505FA5
:1008E00053454354494F4E20343039360A0042555F
:1008F000494C443A20653664313937352D64697284
:100900007479202830303A34343A313020536570CD
:100910002020392032303136290A005649443A2005
:1009200030784645454428742E6D2E6B2E29205074
:1009300049443A203078434146452848484B4220B4
:100940006D6F6429205645523A203078303130346A
:100950000A00444553433A20742E6D2E6B2E206BB3
:100960006579626F617264206669726D7761726524
:1009700020666F722048484B42206D6F640A000A5F
:10098000092D2056657273696F6E202D0A000A6D5D
:100990006F7573653A206F66660A000A6D6F75732E
:1009A000653A206F6E0A000A6B6579626F61726446
:1009B0003A206F66660A000A6B6579626F6172643D
:1009C0003A206F6E0A000A6D61747269783A206F7E
:1009D00066660A000A6D61747269783A206F6E0A61
:1009E000000A64656275673A206F6E0A000A6465E2
:1009F0006275673A206F66660A000A0A626F6F7452
:100A00006C6F616465722E2E2E2000433E20000024
:100A100011241FBECFEFDAE0DEBFCDBF04B603FE68
:100A200027C08091090290910A02A0910B02B09117
:100A30000C028730904BA740B04BD1F410920902C2
:100A400010920A0210920B0210920C0214BE84B78C
:100A5000877F84BF0FB6F894A89580916000886165
:100A600080936000109260000FBEE0E0F8E309950B
:100A700011E0A0E0B1E0E0EBF8E402C005900D92D7
:100A8000A833B107D9F722E0A8E3B1E001C01D9275
:100A9000A930B207E1F70E94AB090C9456240C94DC
:100AA0000000FF93EF93E0913801F0913901309706
:100AB00009F00995EF91FF910895FC01859180302F
:100AC00011F0EFDFFBCF0895FF27E0E230E247FFB0
:100AD0000CC0419597FF09C0EDE260957095809537
:100AE0009095611D711D811D911D27FF02C02195EB
:100AF00030E350E2AA27660F771F881F991FAA1FAD
:100B0000A41710F0A41B63955A95A9F7AA3008F012
:100B1000A95FA05DAF93F3956115710581059105FE
:100B200041F7ED3211F4EF93F395F21718F43F9378
:100B3000F395FBCF8F91B5DFFA95E1F70895E99131
:100B4000F9918591803021F0853219F0AADFF9CF33
:100B5000089520E0E89455915532C1F3503311F4D3
:100B6000689455915A3348F4505390F3220F022E53
:100B7000220F220F200D250FF4CF0EF4219589911D
:100B80009991533619F3533729F1533559F1BC0173
:100B900088279927E8945C3621F489919991689483
:100BA0005591543639F446EF7EF077FF0DC08FEF44
:100BB0009FEF0AC055374AE039F0583540E121F03F
:100BC000523642E009F00895FF93EF937DDFEF91F5
:100BD000FF91B7CFFF93EF93FC0181918030B9F380
:100BE00060DFFBCFFF93EF9368DFF1CFDF93CF930D
:100BF000CDB7DEB72596A3DFCF91DF9108958FEFB4
:100C000084B980E485B957985F9A2E9A2F98E2E4C8
:100C1000F1E088E08E0F11928E13FDCFEAE3F1E050
:100C200088E08E0F11928E13FDCF82E491E09093B5
:100C30004D0180934C018AE391E090934B018093A6
:100C40004A0108950F931F93CF93DF9380914A0138
:100C500090914B0120914C0130914D0130934B010B
:100C600020934A0190934D0180934C01C0E0D0E065
:100C700001E010E080E090E025B1207C2C2BAC015D
:100C800033E0440F551F3A95E1F7242B25B9EAE1EB
:100C9000EA95F1F700C0E0914A01F0914B01EC0FA9
:100CA000FD1F208130E0082E02C0359527950A945B
:100CB000E2F720FD2F9AF5E3FA95F1F70000E6B58B
:100CC0002E982AE12A95F1F700C040914C015091ED
:100CD0004D01DA01AC0FBD1F4F9B0AC09801082ED1
:100CE00001C0220F0A94EAF720953C91232308C003
:100CF0006C919801082E01C0220F0A94EAF7262B66
:100D00002C9326B56E2F70E02E1718F026B530E024
:100D100004C026B530E021503F4F261B370B26304C
:100D2000310558F0E0914A01F0914B01EC0FFD1FA5
:100D30002081FA01EC0FFD1F20833AE13A95F1F78B
:100D400000C02F982E9AEBE2F1E03197F1F700C046
:100D5000000001968830910509F08ECFA0914C01DA
:100D6000B0914D01AC0FBD1FE0914A01F0914B01D4
:100D7000EC0FFD1F9C918081981751F00E946B1B16
:100D800060934E0170934F018093500190935101F5
:100D90002196C830D10509F06DCF809100028530D1
:100DA00021F080910002811111C060914E0170917B
:100DB0004F0180915001909151010E94A11B61311E
:100DC00077428105910510F00E94EE1A81E0DF91D3
:100DD000CF911F910F91089520914C0130914D01B9
:100DE000F901E80FF11D808108950F931F93CF93B0
:100DF000DF938CE291E00E945D05C0E0D0E000E26C
:100E000011E0E0914C01F0914D01EC0FFD1F80814C
:100E10000E94C41A1F928F93DF93CF931F930F9357
:100E20000E94F60521960F900F900F900F900F9053
:100E30000F90C830D10529F7DF91CF911F910F9105
:100E4000089508950895569A81FF02C05E9A089504
:100E50005E9808958091750108959FB7F894109257
:100E600054019FBF90910002943009F057C09091B7
:100E7000E9009F703091EC00232F217030FD20E8B5
:100E8000922B24E02093E9002091EB0020FF43C047
:100E90002091EE0027FF3FC020915201222321F034
:100EA0002091E80025FF37C01092520126E03091D2
:100EB000E80035FD15C030910002343061F5309105
:100EC000EB0035FD28C0215021F481E080935201D0
:100ED00022C0EFE9FFE03197F1F700C00000E7CF53
:100EE0008093F1008091E80085FD0AC08091E800C0
:100EF00080FFFCCF8091E8008E778093E80006C0E9
:100F00008FB7F89421E0209354018FBF9F70909386
:100F1000E90080E008959F709093E9008FEF0895B5
:100F2000CF93DF9300D01F92CDB7DEB79C018091A5
:100F30000002843019F593E099833B832A839093D0
:100F4000E9008FEF9091E800815095FD06C095ED86
:100F50009A95F1F700008111F5CF8091E80085FFA7
:100F60000DC040E050E063E070E0CE0101960E94C9
:100F7000710A8091E8008E778093E8000F900F90BF
:100F80000F90DF91CF910895CF93DF9300D01F9200
:100F9000CDB7DEB720910002243021F522E029836D
:100FA0009B838A8383E08093E9008FEF9091E80030
:100FB000815095FD06C095ED9A95F1F700008111DD
:100FC000F5CF8091E80085FF0DC040E050E063E080
:100FD00070E0CE0101960E94710A8091E8008E7740
:100FE0008093E8000F900F900F90DF91CF910895BC
:100FF000209100022430F1F422E02093E9002FEF49
:101000003091E800215035FD06C035ED3A95F1F7F5
:1010100000002111F5CF2091E80025FF0BC040E032
:1010200050E065E070E00E94710A8091E8008E77E0
:101030008093E8000895CF93DF932091000224303D
:1010400009F048C0EC0180910A018823E1F0809109
:101050000B018823C1F085E08093E9008FEF909128
:10106000E800815095FD06C095E19A95F1F70000E2
:101070008111F5CF8091E80085FF2CC040E050E061
:1010800060E270E017C081E08093E9008FEF9091FB
:10109000E800815095FD06C095ED9A95F1F70000A6
:1010A0008111F5CF8091E80085FF14C040E050E049
:1010B00068E070E0CE010E94710A8091E8008E77AE
:1010C0008093E80080E2FE01A5E5B1E001900D9279
:1010D0008A95E1F7DF91CF91089581E791E00E9431
:1010E0005D058091FF01811109C00E94080C0E94DA
:1010F000650C8091E20084608093E20008958DE6A3
:1011000091E00E945D051092FF01089589E691E04B
:101110000C945D05209153012F5F822F62E30E94A2
:101120001C24992319F02093530108951092530120
:1011300080915401882371F180910002843041F53F
:101140008091E9008F702091EC00922F917020FD2A
:1011500090E8892B94E09093E9009091EB0090FF48
:1011600014C09091EE0097FF10C09091E80095FF99
:1011700003C01092F100F9CF9091E80090FF05C0F4
:101180009091E8009E779093E8008F708093E9003B
:1011900010925401089542E061EC81E00E94820BBC
:1011A00042E061EC82E00E94820B42E061EC83E06D
:1011B0000E94820B42E261EC84E00E94820B42E2D8
:1011C00061EC85E00C94820B80910202833009F47B
:1011D00055C030F4813071F0823009F48EC008952A
:1011E0008A3009F47AC08B3009F460C0893009F084
:1011F0009CC020C080910102813A09F096C0809184
:10120000E800877F8093E8008091050290910602B4
:10121000892B21F460E285E591E003C060E080E085
:1012200090E070E00E94BE0A8091E8008B77809386
:10123000E800089580910102813209F076C0809122
:10124000050290910602009719F0049709F06DC00D
:101250008091E800877F8093E8008091E80082FD1C
:1012600005C0809100028111F8CF5FC08091F1002C
:10127000809375018091E8008B7753C080910102C3
:10128000813A09F052C08091050290910602892BA3
:1012900009F04BC08091E800877F8093E80080913F
:1012A000E80080FFFCCF80910A0136C080910102E6
:1012B0008132D9F58091050290910602892BA9F51A
:1012C0008091E800877F8093E8000E94B70B8091AF
:1012D000030280930A010C944D1480910102813223
:1012E00021F58091E800877F8093E8000E94B70B8A
:1012F0008091040280937601089580910102813AE1
:10130000A1F48091E800877F8093E8008091E80055
:1013100080FFFCCF809176018093F1008091E800FE
:101320008E778093E8000C94B70B08950895089584
:10133000089585E691E00E945D050C9498090E944D
:10134000EE1A8091FE01882329F00E94171B81115B
:101350000C945B0A089584B7877F84BF0FB6F89416
:10136000A895809160008861809360001092600071
:101370000FBE90E080E80FB6F894809361009093E0
:1013800061000FBE0E9496090E944E0F0E94080C39
:101390000E94650C8091E20084608093E2008DE2FF
:1013A00097E00E94BF1A789480910002843019F06F
:1013B0000E94A10EF9CF80E591E00E945D050E9498
:1013C000500F80E091E00E94BC0E8FE391E00E94FC
:1013D0005D050E94970980910002853039F48BE306
:1013E00091E00E945D050E949F09F5CF0E94540F75
:1013F0000E94A10EF0CF0C942B1B81E691E00E947D
:101400005D050C94FB09292F332723303105C9F0E2
:1014100064F42130310581F02230310509F043C0F8
:101420008DE890E02DE931E042C021323105F1F044
:101430002232310541F137C082E190E02AE232E008
:1014400036C099278130910541F08230910541F0F5
:10145000892B49F5E9E9F1E005C0E9E8F1E002C0CE
:10146000E5E7F1E0849190E09F0121C06530D8F478
:10147000E62FF0E0EE0FFF1FED5DFE4F2081318182
:1014800089E090E014C0653070F470E0FB01EE0F6D
:10149000FF1FE75EFE4F20813181FB01EC5EFE4FB6
:1014A000808190E004C080E090E020E030E0FA012C
:1014B00031832083089580E189BD82E189BD09B42B
:1014C00000FEFDCF8091D8008F7D8093D800809161
:1014D000E00082608093E0008091E00081FDFCCF1D
:1014E0000895CF92DF92EF92FF920F931F93CF93C5
:1014F000DF93EC018B017A010E94D60B811135C07C
:10150000E114F10439F0F70180819181081B190B76
:10151000C80FD91FC12CD12C0115110529F18091BB
:10152000E80085FD18C08091E8008E778093E80080
:101530000E94A10EE114F10449F0F701808191812C
:10154000C80ED91ED182C08285E00FC00E94D60B82
:10155000882311F30AC089918093F1000150110989
:10156000FFEFCF1ADF0AD8CF80E0DF91CF911F9134
:101570000F91FF90EF90DF90CF9008952091070298
:10158000309108022617370748F06115710539F4C4
:101590002091E8002E772093E80001C0B90140E0D7
:1015A00061157105A9F120910002222309F443C0BD
:1015B000253009F442C02091E80023FD40C020916D
:1015C000E80022FD32C02091E80020FFE9CF4091E1
:1015D000F3002091F20030E0342BFC01CF016115C3
:1015E000710559F02830310540F481918093F10064
:1015F000615071092F5F3F4FF1CF41E02830310535
:1016000009F040E02091E8002E772093E800C8CF51
:101610004111C9CF0AC080910002882361F0853052
:1016200061F08091E80083FD0AC08091E80082FFAC
:10163000F2CF80E0089582E0089583E0089581E08C
:10164000089520910702309108022617370748F0C5
:101650006115710539F42091E8002E772093E80098
:1016600001C0B901FC0120E06115710591F1809183
:101670000002882309F440C0853009F43FC08091FE
:10168000E80083FD3DC08091E80082FD2FC080917D
:10169000E80080FFE9CF2091F3008091F20090E014
:1016A000922B6115710559F08830910540F4249111
:1016B0002093F1003196615071090196F2CF21E03B
:1016C000089709F020E08091E8008E778093E80089
:1016D000CBCF2111CCCF0AC080910002882361F0CA
:1016E000853061F08091E80083FD0AC08091E800B8
:1016F00082FFF2CF80E0089582E0089583E00895AC
:1017000081E00895982F973058F59093E900981745
:1017100039F07091EC002091ED005091F00003C081
:10172000242F762F50E021FF19C03091EB003E7F2F
:101730003093EB003091ED003D7F3093ED00309120
:10174000EB0031603093EB007093EC002093ED00E0
:101750005093F0002091EE0027FF07C09F5FD3CF8A
:101760008F708093E90081E0089580E00895809172
:10177000010287FF11C08091E80082FD05C08091C1
:1017800000028111F8CF11C08091E8008B770BC067
:1017900080910002882349F08091E80080FFF8CF13
:1017A0008091E8008E778093E80008952091E4000E
:1017B0003091E50095E64091EC00842F817040FF68
:1017C00022C08091E80080FD1CC080910002882327
:1017D00091F0853091F08091EB0085FD10C0409133
:1017E000E4005091E5004217530729F39A01915004
:1017F00011F784E0089582E0089583E0089581E080
:10180000089580E008954091E80042FFDECF0895FA
:101810000E94760C0E947E0CE0EEF0E080818160F8
:101820008083E8EDF0E080818F77808319BCA7ED9D
:10183000B0E08C918E7F8C9380818F7E808310921C
:10184000FF0108950F931F93CF93DF930E94760CAF
:101850000E947E0CC8EDD0E088818F7788838881D4
:101860008068888388818F7D888319BC10920002EC
:101870001092FC011092FE011092FD0100EE10E0AA
:10188000F80180818B7F808388818160888342E03A
:1018900060E080E00E94820BE1EEF0E080818E7FCC
:1018A0008083E2EEF0E080818160808380818860C7
:1018B0008083F80180818E7F808388818061888326
:1018C000DF91CF911F910F910895E8EDF0E08081B5
:1018D0008F7E8083E7EDF0E080818160808384E00B
:1018E00082BF81E08093FF010C94220CE8EDF0E0D0
:1018F00080818E7F80831092E20008951092DA003A
:101900001092E10008951F920F920FB60F921124CA
:101910002F933F934F935F936F937F938F939F93F7
:10192000AF93BF93EF93FF938091E10082FF0BC0D1
:101930008091E20082FF07C08091E1008B7F80935D
:10194000E1000E948A088091DA0080FF1FC0809128
:10195000D80080FF1BC08091DA008E7F8093DA0070
:101960008091D90080FF0DC080E189BD82E189BDF1
:1019700009B400FEFDCF81E0809300020E946D0853
:1019800005C019BC109200020E947F088091E100FE
:1019900080FF19C08091E20080FF15C08091E200B5
:1019A0008E7F8093E2008091E20080618093E2006C
:1019B0008091D80080628093D80019BC85E0809324
:1019C00000020E9499098091E10084FF30C080915B
:1019D000E20084FF2CC080E189BD82E189BD09B4A9
:1019E00000FEFDCF8091D8008F7D8093D80080913C
:1019F000E1008F7E8093E1008091E2008F7E8093F2
:101A0000E2008091E20081608093E2008091FC011D
:101A1000882311F084E007C08091E30087FD02C0B5
:101A200081E001C083E0809300020E94FD09809163
:101A3000E10083FF24C08091E20083FF20C08091F9
:101A4000E100877F8093E10082E0809300021092A2
:101A5000FC018091E1008E7F8093E1008091E200A3
:101A60008E7F8093E2008091E20080618093E200AB
:101A700042E060E080E00E94820B0E948608FF91B5
:101A8000EF91BF91AF919F918F917F916F915F91F6
:101A90004F913F912F910F900FBE0F901F9018956F
:101AA0001F93CF93DF93CDB7DEB7AA970FB6F89405
:101AB000DEBF0FBECDBFE1E0F2E088E08E0F909177
:101AC000F10091938E13FBCF0E94E4088091E8000F
:101AD00083FF1FC18091010290910202492F50E0C3
:101AE0004A30510508F015C1FA01EA5AFF4F0C942B
:101AF0003C24803881F0823809F00BC180910502C6
:101B00008F708093E9008091EB0085FB882780F936
:101B10001092E90006C08091FD019091FE019111A3
:101B200082609091E800977F9093E8008093F100A5
:101B30001092F100C8C0282F2D7F09F0EAC0882339
:101B400019F0823061F0E5C080910302813009F024
:101B5000E0C0933009F080E08093FE012BC08091BB
:101B60000302811127C0809105028F7009F4D1C052
:101B70008093E9002091EB0020FF1CC0933021F4FA
:101B80008091EB00806214C09091EB009061909383
:101B9000EB0021E030E0A90102C0440F551F8A95F7
:101BA000E2F74093EA001092EA008091EB0088602F
:101BB0008093EB001092E9008091E800877F86C057
:101BC0008111A7C0109103021F778091E3008078F4
:101BD000812B8093E3008091E800877F8093E80069
:101BE0000E94B70B8091E80080FFFCCF8091E3005A
:101BF00080688093E300111102C082E001C083E09D
:101C00008093000286C08058823008F082C08091A4
:101C10000302909104028C3D53E0950779F583E02F
:101C20008A838AE289834FB7F894DE01139620E015
:101C30003EE051E2E32FF0E050935700E49120FFA3
:101C400003C0E295EF703F5FEF708E2F90E0EA30B7
:101C500010F0C79601C0C0968D939D932F5F2431DD
:101C600049F74FBF8091E800877F8093E8006AE2E0
:101C700070E0CE0101960E94BE0A14C0AE014F5F13
:101C80005F4F609105020E94030ABC01892B09F491
:101C900040C09091E800977F9093E80089819A81F5
:101CA0000E94210B8091E8008B778093E80031C07F
:101CB000803879F58091E800877F8093E8008091F3
:101CC000FC018093F1008091E8008E778093E8001A
:101CD0000E94B70B1EC081111CC09091030292306C
:101CE000C0F48091E800877F8093E8009093FC0126
:101CF0000E94B70B8091FC01811106C08091E30026
:101D000087FD02C081E001C084E0809300020E9450
:101D1000CB088091E80083FF0AC08091E800877FAC
:101D20008093E8008091EB0080628093EB00AA969C
:101D30000FB6F894DEBF0FBECDBFDF91CF911F91DC
:101D40000895CF93809100028823A1F0C091E9000B
:101D5000CF709091EC00892F817090FD80E8C82BA6
:101D60001092E9008091E80083FD0E94500DCF7031
:101D7000C093E900CF91089590937C0180937B01FB
:101D80000895E0917B01F0917C01309721F0019062
:101D9000F081E02D099480E00895EF92FF920F9377
:101DA0001F93CF93DF93E0917B01F0917C013097FB
:101DB000B1F18C010280F381E02D09958091EB0156
:101DC00082FF2DC080FF04C082E693E00E945D0583
:101DD000E80110E28CE5E82E83E0F82E8091EB011B
:101DE00080FF0BC088811F928F93FF92EF920E9419
:101DF000F6050F900F900F900F9011502196111132
:101E0000EDCF8091EB0180FF0AC08AE593E0DF917E
:101E1000CF911F910F91FF90EF900C945D05DF9192
:101E2000CF911F910F91FF90EF900895E0917B016A
:101E3000F0917C01309721F00480F581E02D099428
:101E400008952091790130917A018217930771F0FA
:101E500090937A0180937901E0917B01F0917C016C
:101E6000309721F00680F781E02D099408952091A4
:101E70007701309178018217930771F09093780180
:101E800080937701E0917B01F0917C01309721F004
:101E90000084F185E02D0994089508950C944D0F68
:101EA0000E94561B0C94FF05CF92DF92EF92FF9297
:101EB0000F931F93CF93DF9300D000D000D0CDB706
:101EC000DEB70E9422068EE7C82E81E0D82E00E001
:101ED00010E0E02E802F0E94EC06F60141916F0188
:101EE000F42EF826B1F40F5F1F4F0830110589F763
:101EF0008FEF89838A831B820E945F1B8160782F0A
:101F00009D838C8349815A816B818D810E9413103E
:101F100047C09091EB0191FF04C08E830E94F506AB
:101F20008E8120E030E04F2D50E0922FBA01022E3A
:101F300002C0759567950A94E2F760FF2BC029836C
:101F4000EA8221E030E0690102C0CC0CDD1C9A95E8
:101F5000E2F790E08C219D21892B09F420E02B836E
:101F60000E945F1B8160782F9D838C8349815A81F9
:101F70006B818D810E94131049815A816B817C8114
:101F80008D810E94DB1AF801E258FE4F8081C8263D
:101F9000C08206C02F5F3F4F2830310531F6A3CFF6
:101FA0000E94DA1A0E944C1E10917D010E94C10EFF
:101FB000181741F10E94C10E80937D019091EB01B1
:101FC00092FF0EC090FF0CC01F928F9384E793E0A6
:101FD0009F938F930E94F6050F900F900F900F9094
:101FE00080917D0126960FB6F894DEBF0FBECDBF5F
:101FF000DF91CF911F910F91FF90EF90DF90CF90E5
:102000000C94EC1A26960FB6F894DEBF0FBECDBF27
:10201000DF91CF911F910F91FF90EF90DF90CF90C4
:1020200008950C942307CF93DF93CDB7DEB72B979A
:102030000FB6F894DEBF0FBECDBF942F4F83252F70
:10204000588769877A878B874A855B85452B21F07E
:102050002F3F09F59F3FF9F4DE01119686E0FD015F
:1020600011928A95E9F785E0FE01379601900D926D
:102070008A95E1F749815A816B817C818D819E81AE
:102080000E94F0162B960FB6F894DEBF0FBECDBFA0
:10209000DF91CF9108954F81588569857A858B8529
:1020A0000E94DB1AD9CFCF93882309F4A4C0C82F8C
:1020B0008CEF8C0F813A48F48C2F0E94962181116D
:1020C0009AC08C2F0E947B190CC080E28C0F883044
:1020D00058F4C77081E001C0880FCA95EAF70E94E2
:1020E000261ACF910C946A1A8BE58C0F833078F402
:1020F000C53A29F0C63A31F083E890E005C081E89E
:1021000090E002C082E890E0CF910C94210F88E526
:102110008C0F853108F06FC0C83A61F1C93A69F196
:10212000CA3A71F1CB3A79F1CC3A81F1CD3A89F1E1
:10213000CE3A91F1CF3A99F1C13BA1F1C03BA9F15F
:10214000C23BB1F1C33BB9F1C43BC1F1C53BC9F1DD
:10215000C63BD1F1C73BD9F1C83BE1F1C93BE9F13D
:10216000CA3BF1F1CB3BF9F1CC3B09F43FC080E035
:1021700090E03EC082EE90E03BC089EE90E038C037
:102180008AEE90E035C085EB90E032C086EB90E0BF
:102190002FC083EB90E02CC084EB90E029C087EB4C
:1021A00090E026C08CEC90E023C08DEC90E020C045
:1021B00083E891E01DC08AE891E01AC082E991E0CD
:1021C00017C084E991E014C081E292E011C083E27B
:1021D00092E00EC084E292E00BC085E292E008C07B
:1021E00086E292E005C087E292E002C08AE292E0D5
:1021F000CF910C94370FCF910895882329F19CEF4C
:10220000980F913A18F40E94CE190DC090E2980FE1
:10221000983058F4877091E001C0990F8A95EAF7D9
:10222000892F0E942C1A0C946A1A9BE5980F933000
:1022300020F480E090E00C94210F885A853120F43E
:1022400080E090E00C94370F0895882321F00E94DD
:10225000261A0C946A1A0895882321F00E942C1AD9
:102260000C946A1A0895CF92DF92EF92FF920F9327
:102270001F93CF93DF9300D000D000D0CDB7DEB74F
:1022800025E0FC01DE01119601900D922A95E1F7FF
:10229000FC0140813181F280258122952F7063817C
:1022A0007481672B09F4D8C23F3F19F44F3F09F4FA
:1022B000D3C26C0149833A8389819A812E830E941B
:1022C0003A19182F092F0E9439190E944918E02F36
:1022D000E295EF70F0E0E05AFF4F2E810C943C2421
:1022E000802F807F902F9F70092F882311F00295F7
:1022F000007FFF2049F0002309F45FC2802F0E9475
:10230000391A0E946A1A59C2812F0E94FD100023B7
:1023100009F4A2C2802F0E943F1A26960FB6F894A5
:10232000DEBF0FBECDBFDF91CF911F910F91FF9008
:10233000EF90DF90CF900C946A1A802F807F902FBF
:102340009F70092F803211F00295007F112319F040
:10235000113001F129C0FF20A9F0802F222349F17B
:10236000213039F526960FB6F894DEBF0FBECDBFEB
:10237000DF91CF911F910F91FF90EF90DF90CF9061
:102380000C94491A222319F0213009F465C20E94E5
:10239000521A2CC0FF20E9F0263008F05DC20E94DE
:1023A000231A802329F022C0FF20F1F0211115C04B
:1023B000802F26960FB6F894DEBF0FBECDBFDF91FB
:1023C000CF911F910F91FF90EF90DF90CF900C94E1
:1023D0002511253008F040C209C0F601858180FF33
:1023E000ECC18F708583E4CF2111FBC1802F69C1BF
:1023F000202F26952695237030E02115310521F0F8
:1024000021303105C9F028C2FF2021F0812F902F03
:10241000937002C080E090E026960FB6F894DEBF7D
:102420000FBECDBFDF91CF911F910F91FF90EF9025
:10243000DF90CF900C94210FFF2021F0812F902F5F
:10244000937002C080E090E026960FB6F894DEBF4D
:102450000FBECDBFDF91CF911F910F91FF90EF90F5
:10246000DF90CF900C94370F812FFF2019F00E943E
:10247000D21C02C00E943A1D26960FB6F894DEBF09
:102480000FBECDBFDF91CF911F910F91FF90EF90C5
:10249000DF90CF900C94BF1D802F837009F078C01F
:1024A000F110DAC1812F829586958770880F880F89
:1024B000912F9F70C92ED12CE12CF12C082E04C035
:1024C000CC0CDD1CEE1CFF1C0A94D2F714FF12C0CA
:1024D0004FE050E060E070E004C0440F551F661FFD
:1024E000771F8A95D2F7CB01BA01609570958095D8
:1024F000909503C060E070E0CB01202F26952695D3
:102500002370422F50E042305105D1F04330510545
:1025100059F16C297D298E299F294130510541F1BE
:1025200026960FB6F894DEBF0FBECDBFDF91CF91D8
:102530001F910F91FF90EF90DF90CF900C945E1859
:102540006C297D298E299F2926960FB6F894DEBF27
:102550000FBECDBFDF91CF911F910F91FF90EF90F4
:10256000DF90CF900C9470180E945E18C701B601DE
:1025700026960FB6F894DEBF0FBECDBFDF91CF9188
:102580001F910F91FF90EF90DF90CF900C944C181B
:10259000FF2019F0802F817001C08695882309F4EF
:1025A0005BC1812F829586958770880F880F912F48
:1025B0009F70C92ED12CE12CF12C082E04C0CC0C1C
:1025C000DD1CEE1CFF1C0A94D2F714FF12C04FE072
:1025D00050E060E070E004C0440F551F661F771F95
:1025E0008A95D2F7CB01BA01609570958095909548
:1025F00003C060E070E0CB01202F26952695237064
:10260000422F50E042305105D1F04330510559F18D
:102610006C297D298E299F294130510541F126964B
:102620000FB6F894DEBF0FBECDBFDF91CF911F91E3
:102630000F91FF90EF90DF90CF900C9415196C29BB
:102640007D298E299F2926960FB6F894DEBF0FBEEE
:10265000CDBFDF91CF911F910F91FF90EF90DF9051
:10266000CF900C9427190E941519C701B601269620
:102670000FB6F894DEBF0FBECDBFDF91CF911F9193
:102680000F91FF90EF90DF90CF900C940319103FC3
:1026900041F118F4103E48F48BC0123F09F450C0C9
:1026A000D8F1133F09F460C083C01F70802F8F7171
:1026B000FF2021F00E949C18812F7BCE0E94BD1824
:1026C000812F26960FB6F894DEBF0FBECDBFDF91E7
:1026D000CF911F910F91FF90EF90DF90CF900C94CE
:1026E0002C11FF20A9F0253008F0B6C0802F8F7183
:1026F00026960FB6F894DEBF0FBECDBFDF91CF9107
:102700001F910F91FF90EF90DF90CF900C94E21803
:10271000263008F0A1C0EACFFF20A1F0802F8F71F2
:1027200026960FB6F894DEBF0FBECDBFDF91CF91D6
:102730001F910F91FF90EF90DF90CF900C949C1819
:10274000FF2061F3802F8F7126960FB6F894DEBFBD
:102750000FBECDBFDF91CF911F910F91FF90EF90F2
:10276000DF90CF900C94BD18FF2091F0802F8F71D7
:1027700026960FB6F894DEBF0FBECDBFDF91CF9186
:102780001F910F91FF90EF90DF90CF900C948718DE
:1027900026960FB6F894DEBF0FBECDBFDF91CF9166
:1027A0001F910F91FF90EF90DF90CF900C948218C3
:1027B000FF20A1F0222309F4B1CF812F26960FB676
:1027C000F894DEBF0FBECDBFDF91CF911F910F9167
:1027D000FF90EF90DF90CF900C945310222309F4D8
:1027E000B1CF812F26960FB6F894DEBF0FBECDBFB6
:1027F000DF91CF911F910F91FF90EF90DF90CF90DD
:102800000C94FD10402F4F70612FC6010E944C1C8C
:1028100026960FB6F894DEBF0FBECDBFDF91CF91E5
:102820001F910F91FF90EF90DF90CF900C94941731
:10283000402F4F70612FC60126960FB6F894DEBF69
:102840000FBECDBFDF91CF911F910F91FF90EF9001
:10285000DF90CF900C944F1C26960FB6F894DEBFF5
:102860000FBECDBFDF91CF911F910F91FF90EF90E1
:10287000DF90CF9008950E94461A0E94151A0E9478
:102880006A1A0E94F11E0E94BF1D80E090E00E9423
:10289000210F80E090E00C94370F0E94361A0C94C0
:1028A0003B140E943A19292F22952F7030E02C30CA
:1028B00031054CF42A3031056CF4225031092230B4
:1028C000310588F407C02C30310549F02F3031052F
:1028D00031F009C0803E48F0803F29F406C093FBE8
:1028E000882780F9089580E0089581E00895CF93C6
:1028F000DF9300D000D01F92CDB7DEB70F900F90BE
:102900000F900F900F90DF91CF910895CF93DF93A9
:1029100000D000D000D0CDB7DEB726960FB6F89421
:10292000DEBF0FBECDBFDF91CF9108951F93CF9330
:10293000DF93C091860116E080918701C81799F056
:10294000D0E01C9FF0011D9FF00D1124E857FE4FB1
:102950004081518162817381848195810E948614B6
:102960002196C770E9CFDF91CF911F9108954091D3
:10297000B8015091B9016091BA017091BB01809189
:10298000BC019091BD010C9486148091BD0182958B
:102990008F7009F054C08091BA01882309F44FC0A8
:1029A00080918601A09187016091B8017091B90171
:1029B0004091BB015091BC01B6E08A1709F43FC0B9
:1029C00090E041155105C1F17F3F11F46F3FA1F136
:1029D000B89FF001B99FF00D1124E857FE4F2181F7
:1029E00072132AC02081621327C02281211124C0C2
:1029F000238134812417350710F421503109241B19
:102A0000350B2C323140C0F42091BD012F70206174
:102A10002093BD0126E0289FF001299FF00D11248D
:102A2000E357FE4F80818F708061808388EB91E057
:102A30000E9433110C94961401968770BECF0895AE
:102A4000CF92DF92EF92FF920F931F93CF93DF937A
:102A5000CDB7DEB762970FB6F894DEBF0FBECDBF1D
:102A60008C0185E0F801DE011D9601900D928A959A
:102A7000E1F7D8014C9111965C91119712966C91E7
:102A800012971396CD90DC9014973091B801709105
:102A9000B9018091BB019091BC01009709F473C109
:102AA0007F3F19F43F3F09F46EC1E090BA01EE2078
:102AB00009F4C5C02091BD01C816D90650F0F60131
:102AC000E81BF90BCF01FF24F3948C329140C8F03E
:102AD00009C0809590958C0D9D1DFF24F3948C3238
:102AE000914078F0F12C207F09F0C6C07C2DD98A66
:102AF000C88A89890E94771488EB91E00E9433117B
:102B0000B1C0822F807F09F045C0751313C0341304
:102B100011C061110FC02F7020612093BD010E9470
:102B2000B71488EB91E00E9433118091BD01F80148
:102B300085832EC0CD2819F15F3F11F44F3FF9F086
:102B4000F62E61111CC0809186012091870136E02C
:102B5000821709F45BC090E0389FF001399FF00DB7
:102B60001124E857FE4F7181571306C07081471337
:102B700003C07281711103C001968770E9CFF62EF0
:102B8000662309F41DC18091BD0181608093BD0160
:102B9000F12C16C1751309C0341307C0611105C0AB
:102BA0008091BD01F8018583C8C04D875E878D8502
:102BB0009E856A8B0E9451146A898823E1F16623FD
:102BC000D1F12091BD01822F82958F7090E0029704
:102BD00074F08091B8019091B90198878F8319861C
:102BE000DB86CA862C87CE0107960E94331186E0C9
:102BF000F801A8EBB1E001900D928A95E1F70E94EF
:102C0000C5140E94B714FF24F394DAC04D875E8781
:102C10008D859E850E943A19292F22952F7030E0CC
:102C2000223031050CF0BFC09F7009F0B9C0805E42
:102C3000883008F4C5C0C8010E943311E4CFC8161B
:102C4000D90608F453C0F601E81BF90BCF018C320A
:102C5000914008F453C0F12C7C2DD98AC88A898907
:102C60000E947714E8EBF1E086E0DF011D928A957F
:102C7000E9F70E94B714A4C0751314C0341312C02E
:102C8000611110C08091BD01F8018583C8010E94C7
:102C9000331186E0E8EBF1E0DF011D928A95E9F758
:102CA000FE2C8EC04D875E878D859E856A8B0E9427
:102CB00051146A89882309F4BECF662309F4BBCF77
:102CC0002091BD01822F82958F7090E002970CF4C5
:102CD0008ECF8091B8019091B9019A8389831B822C
:102CE000DD82CC822E83CE0101967FCF8095909598
:102CF0008C0D9D1D8C32914008F0ADCFF62E6623D1
:102D000009F499CF75132EC034132CC02091BD0146
:102D100020FD1FC0822F82958F70D9F0D8011596A3
:102D20002C9315978F3049F08F5F982F9295907F55
:102D3000822F8F70892B15968C93C8010E943311B6
:102D400086E0F801A8EBB1E001900D928A95E1F7D9
:102D500090CF86E0F801A8EBB1E001900D928A9542
:102D6000E1F72EC04D875E878D859E850E945114A8
:102D700081113DCF8091BD0181608093BD01C8016B
:102D80000E9433111DC0662309F455CF4D875E871D
:102D90008D859E850E945114882309F44CCF27CF3E
:102DA000811145CF0DC0243031050CF044CF9F7008
:102DB00009F43DCFD80115969C91907F09F037CF4B
:102DC0008F2D62960FB6F894DEBF0FBECDBFDF9198
:102DD000CF911F910F91FF90EF90DF90CF900895CA
:102DE0001F93CF93DF93CDB7DEB72C970FB6F89430
:102DF000DEBF0FBECDBF4F83588769877A878B8729
:102E00009C87CE0107960E942015882369F08F8148
:102E100098852A853B85232BF1F19F3F09F063C0FC
:102E20008F3F09F060C037C086E0FE013796DE01B3
:102E3000119601900D928A95E1F76F817885EA8568
:102E4000FB85309741F17F3F11F46F3F21F12091D5
:102E5000870130E0C901019687709927409186016A
:102E600050E08417950709F447C069837A83FD838E
:102E7000EC8396E0929FD001939FB00D1124A85748
:102E8000BE4FFE01319601900D929A95E1F7809325
:102E900087010E94961416E0809186019091870127
:102EA0008917C1F1189FC001112488579E4F0E94B5
:102EB0002015882379F1E09186011E9FF0011124ED
:102EC000E857FE4F408151816281738184819581F1
:102ED0000E9486148091860190E001968770992760
:102EE00080938601D9CF4F81588569857A858B85F6
:102EF0009C850E948614CFCF0E944D1410928701AA
:102F000010928601E8EBF1E086E0DF011D928A95E0
:102F1000E9F7C1CF2C960FB6F894DEBF0FBECDBF38
:102F2000DF91CF911F910895DF92EF92FF920F935F
:102F30001F93CF93DF93FC01892B09F48AC0E12C06
:102F4000F12CDD24D394EF0121968491853709F487
:102F500061C058F4843708F04EC0843008F06AC06D
:102F60008130D1F0823071F174C0883709F45DC0CE
:102F700050F4863709F455C0873709F06AC08E2DA2
:102F80000E94331A54C09CE7980F903708F061C034
:102F90008F770E94FD1050C08F010E5F1F4FFE0102
:102FA000849190E2980F983050F48770FD2D01C005
:102FB000FF0F8A95EAF78F2F0E94391A14C00E94DA
:102FC000531013C08F010E5F1F4FFE01C49180E2AA
:102FD0008C0F883060F4C7708D2D01C0880FCA95A2
:102FE000EAF70E943F1A0E946A1AE80125C08C2F56
:102FF0000E94FD10FACF9F012E5F3F4FFE01C4914A
:10300000CC2369F08FE99FE00197F1F700C0000041
:10301000C150F6CF9F012E5F3F4FFE01F490E901B2
:103020000BC00E94231AE82E07C00E94361A0E9485
:103030006A1A02C00E9453108F2D882341F0EFE9D5
:10304000FFE03197F1F700C000008150F6CFFE019C
:103050007ACFDF91CF911F910F91FF90EF90DF908A
:1030600008956093C2017093C3018093C40190934B
:10307000C5010E94EA1A0C943B146093BE01709340
:10308000BF018093C0019093C1010E94EB1A0C9480
:103090003B1408950C9431180F931F930091C201B3
:1030A0001091C3012091C4013091C501602B712B97
:1030B000822B932B1F910F910C9431180F931F9318
:1030C0000091C2011091C3012091C4013091C5014A
:1030D00060237123822393231F910F910C94311845
:1030E0000F931F930091C2011091C3012091C4015D
:1030F0003091C50160277127822793271F910F9177
:103100000C94311860E070E0CB010C943D180F93E3
:103110001F9341E050E060E070E08A019B0104C031
:10312000000F111F221F331F8A95D2F7C901B80162
:103130001F910F910C943D180F931F9341E050E0A5
:1031400060E070E004C0440F551F661F771F8A952A
:10315000D2F78091BE019091BF01A091C001B091C2
:10316000C1018A019B01082B192B2A2B3B2BC9017A
:10317000B8011F910F910C943D180F931F9341E0DC
:1031800050E060E070E004C0440F551F661F771FD9
:103190008A95D2F740955095609570958091BE01C3
:1031A0009091BF01A091C001B091C1018A019B0122
:1031B000082319232A233B23C901B8011F910F912A
:1031C0000C943D180F931F9341E050E060E070E0D5
:1031D00004C0440F551F661F771F8A95D2F7809150
:1031E000BE019091BF01A091C001B091C1018A01BF
:1031F0009B01082719272A273B27C901B8011F91DE
:103200000F910C943D180F931F930091BE011091E4
:10321000BF012091C0013091C101602B712B822B25
:10322000932B1F910F910C943D180F931F930091B6
:10323000BE011091BF012091C0013091C1016023F6
:103240007123822393231F910F910C943D180F93A8
:103250001F930091BE011091BF012091C0013091D8
:10326000C10160277127822793271F910F910C942A
:103270003D180895CF92DF92EF92FF920F931F9324
:10328000CF93DF938C01C090C201D090C301E09036
:10329000C401F090C5014091BE015091BF01609101
:1032A000C0017091C101C42AD52AE62AF72ACFE1CC
:1032B000D0E0D701C6010C2E04C0B695A79597950E
:1032C00087950A94D2F780FF07C0B8018C2F0E941F
:1032D000221C8130910531F4219758F7B80180E024
:1032E0000E94221CDF91CF911F910F91FF90EF90D0
:1032F000DF90CF90089590910A01992321F0909149
:103300000B01911109C020910C0130910D01F901BF
:1033100032969FEF40E030C0982F969596959695FF
:103320009F31A0F4E0910C01F0910D01E90FF11D26
:10333000877021E030E0A90102C0440F551F8A9533
:10334000E2F7CA019181892B818308959091EB0165
:1033500090FF23C01F928F938DE993E09F938F93EB
:103360000E94F6050F900F900F900F9008959F3FC9
:1033700039F04F5F4E3141F051915813F8CF0DC0E5
:103380005111F7CF942FF5CF9F3F39F0F901E90F95
:10339000F11D97FDFA9582830895089590910A0191
:1033A000992321F090910B01911109C020910C01FA
:1033B00030910D01F9013296205E3F4F30C0982FB9
:1033C0009695969596959F31A8F4E0910C01F09111
:1033D0000D01E90FF11D877021E030E0A90102C065
:1033E000440F551F8A95E2F7CA0180959181892380
:1033F000818308959091EB0190FF16C01F928F93E7
:103400008FE793E09F938F930E94F6050F900F90A4
:103410000F900F9008953196E217F30729F09081ED
:103420009813F9CF1082F7CF089581E090E0E091F2
:103430000C01F0910D01E80FF91F10820196803206
:103440009105A9F708958091EA0108959091EA0104
:10345000892B8093EA01089580959091EA01892350
:103460008093EA0108958093EA0108951092EA0199
:1034700008959091E901892B8093E9010895809541
:103480009091E90189238093E90108951092E9015F
:1034900008958093C8010E945F1B9093C701809399
:1034A000C60108951092C8011092C7011092C6017A
:1034B000089580910C0190910D01FC0131969C01C1
:1034C000205E3F4F80E0919191118F5FE217F307EB
:1034D000D1F70895E0910C01F0910D018091EA017E
:1034E0008083E0910C01F0910D0190818091E901C0
:1034F000892B80838091C8018823D9F10E945F1BAA
:103500002091C6013091C7018217930748F00E94AD
:103510005F1B2091C6013091C701821B930B0AC02B
:103520000E945F1B2091C6013091C7012095309504
:10353000820F931F8C32914070F08091EB0180FFDD
:1035400008C08BEB93E09F938F930E94F6050F903A
:103550000F900E94521AE0910C01F0910D019081A0
:103560008091C801892B80830E94591A81110E9481
:10357000521A80910C0190910D010C94CD0E9093F4
:1035800039018093380108958295982F9C7C392FBA
:1035900036953695282F237344E0249FC0011124CB
:1035A000932F982B292F2A7A2695892F8575880F96
:1035B000822B08950895CF93DF9300D000D01F92FF
:1035C000CDB7DEB70F900F900F900F900F90DF9157
:1035D000CF910895089508950C94111080910002E0
:1035E000843021F11092EC0120E488E190E00FB6E4
:1035F000F894A895809360000FBE2093600083B775
:10360000817F846083BF83B7816083BF789488950E
:1036100083B78E7F83BF0FB6F894A8958091600022
:10362000886180936000109260000FBE0895CF9370
:103630000E9421070E9422060E942207C0E08C2FD0
:103640000E94EC06811104C0CF5FC830C1F701C0F1
:1036500081E0CF9108950C944D141F920F920FB6F4
:103660000F9211248F939F93AF93BF938091EC019E
:10367000811113C08091ED019091EE01A091EF01B5
:10368000B091F0014196A11DB11D8093ED01909381
:10369000EE01A093EF01B093F001BF91AF919F9124
:1036A0008F910F900FBE0F901F90189582E084BDF0
:1036B00093E095BD9AEF97BD80936E0008952FB764
:1036C000F8948091ED019091EE01A091EF01B091FD
:1036D000F0012FBF08952FB7F8946091ED0170911C
:1036E000EE018091EF019091F0012FBF0895CF92EC
:1036F000DF92EF92FF920F931F932FB7F8944091B0
:10370000ED015091EE016091EF017091F0012FBF3A
:103710006A017B01EE24FF248C0120E030E0C0161A
:10372000D106E206F30610F4415051099A01281B14
:10373000390BC9011F910F91FF90EF90DF90CF904F
:103740000895CF92DF92EF92FF920F931F932FB7BE
:10375000F894C090ED01D090EE01E090EF01F09070
:10376000F0012FBF97018601061B170B280B390BA1
:10377000C616D706E806F90618F0C901B80106C052
:10378000C901B80161507109810991091F910F9117
:10379000FF90EF90DF90CF9008951F920F920FB699
:1037A0000F9211248F939F93AF93BF938091ED015C
:1037B0009091EE01A091EF01B091F0010196A11D51
:1037C000B11D8093ED019093EE01A093EF01B093B2
:1037D000F001BF91AF919F918F910F900FBE0F900D
:1037E0001F9018950E94080CF8942FEF87EA91E635
:1037F000215080409040E1F700C0000087E090EB4E
:10380000DC018093090290930A02A0930B02B0930B
:103810000C029CE088E10FB6F894A89580936000B4
:103820000FBE90936000FFCF28E0929FF00111241B
:10383000E80FF11DE052FF4F9491892F8F70929500
:103840009F700895CF93C82FCB010E94141C282F7E
:1038500030E080E1989FA0011124422B532B403887
:10386000510519F480E090E015C09770E92FF0E061
:1038700088E0C89FE00DF11D112484E0EE0FFF1FCA
:103880008A95E1F7E20FF31FEE0FFF1FE050F849B2
:1038900085919491CF91089580E090E008950895E6
:1038A0008091F30180FF0BC06091110185E0689F5A
:1038B000B001112475956795759567952BC081FFAB
:1038C00009C06091110185E0689FB00111247595D0
:1038D000679520C082FF07C06091110185E0689F55
:1038E000B001112417C09091F4019923D1F0609197
:1038F0001001961788F72091110185E0289F90010B
:103900001124929FA001939F500D112470E0CA01D1
:103910000E9428246038710540F46115710539F062
:1039200002C065E070E0862F08958FE7089581E07A
:1039300008958091F30180FF08C060910F0170E04D
:10394000759567957595679521C081FF06C0609153
:103950000F0170E07595679519C082FF04C06091F2
:103960000F0170E010C09091F4019923C1F06091B3
:103970000E019617A0F780910F01899FC0011124B5
:1039800070E00E9428246038710528F461157105E3
:1039900021F0862F08958FE7089581E0089561E072
:1039A00070E0F4CF803F21F40E94501C819504C048
:1039B000813F29F40E94501C8093F7010895823FB3
:1039C00021F40E94501C819504C0833F29F40E9479
:1039D000501C8093F6010895893F19F40E94991CA8
:1039E00005C08A3F31F40E94991C81958093F801AB
:1039F00008958B3F21F40E94991C819504C08C3F4F
:103A000029F40E94991C8093F9010895843F21F4C0
:103A10008091F501816017C0853F21F48091F50107
:103A2000826011C0863F21F48091F50184600BC053
:103A3000873F21F48091F501886005C0883F31F40B
:103A40008091F50180618093F50108958D3F21F407
:103A50008091F30181600BC08E3F21F48091F301CE
:103A6000826005C08F3F29F48091F30184608093C8
:103A7000F3010895803F39F48091F70187FF6CC00E
:103A80001092F70169C0813F29F48091F70118165F
:103A9000BCF362C09091F601823F29F497FF5CC0AD
:103AA0001092F60159C0833F19F41916CCF354C093
:103AB000893F41F48091F80118160CF04DC0109226
:103AC000F8014AC08A3F29F48091F80187FF44C079
:103AD000F6CF8B3F39F48091F90187FF3DC01092FA
:103AE000F9013AC08C3F29F48091F9011816BCF312
:103AF00033C0843F21F48091F5018E7F17C0853F4C
:103B000021F48091F5018D7F11C0863F21F48091D1
:103B1000F5018B7F0BC0873F21F48091F501877FF2
:103B200005C0883F31F48091F5018F7E8093F501C7
:103B300013C08D3F21F48091F3018E7F0BC08E3F27
:103B400021F48091F3018D7F05C08F3F29F480918E
:103B5000F3018B7F8093F3018091F60181110EC0F8
:103B60008091F70181110AC08091F801811106C08E
:103B70008091F901811102C01092F40108958091A1
:103B8000EB0183FF7EC084EF93E00E945D0580918E
:103B9000F5011F928F938FEE93E09F938F930E9476
:103BA000F6058DEE93E00E945D058091F601282FC9
:103BB000082E000C330B3F938F938AEE93E09F9374
:103BC0008F930E94F60588EE93E00E945D05809138
:103BD000F701282F082E000C330B3F938F9385EEAF
:103BE00093E09F938F930E94F60583EE93E00E94EB
:103BF0005D058091F801282F082E000C330B3F93B0
:103C00008F9380EE93E09F938F930E94F6058EED45
:103C100093E00E945D058091F901282F082E000C89
:103C2000330B3F938F938BED93E09F938F930E9481
:103C3000F60588ED93E00E945D058091F4011F92E6
:103C40008F9385ED93E09F938F930E94F60583ED0C
:103C500093E00E945D058091F3011F928F9380EDA8
:103C600093E09F938F930E94F6058DEC93E00E9462
:103C70005D058DB79EB74C960FB6F8949EBF0FBEEC
:103C80008DBF85EF91E00E94160F0E945F1B9093FD
:103C9000F2018093F10108951F93CF93DF938091F8
:103CA000F1019091F2010E94771BAC019091F40117
:103CB000992321F02091120130E006C020911301D8
:103CC0008AE0289F900111244217530708F485C009
:103CD0008091F601C091F701D091F8011091F9019E
:103CE000811107C0C11175C0D11173C0111171C00C
:103CF00074C09F3F19F09F5F9093F401181624F44D
:103D00000E94501C8093F6018091F60187FF05C048
:103D10000E94501C81958093F6011C1624F40E9489
:103D2000501C8093F7018091F70187FF05C00E9426
:103D3000501C81958093F7016091F601662331F163
:103D4000C091F701CC2311F1062E000C770B880BE4
:103D5000990B0E94232323E333E343E35FE30E94B1
:103D600087230E94EB226093F6016C2FCC0F770B18
:103D7000880B990B0E94232323E333E343E35FE3A0
:103D80000E9487230E94EB226093F7011D1624F402
:103D90000E94991C8093F8018091F80187FF05C06B
:103DA0000E94991C81958093F801111624F40E94B9
:103DB000991C8093F9018091F90187FF05C00E9449
:103DC000991C81958093F901DF91CF911F910C94FB
:103DD000BF1D9F3F09F08FCF97CFDF91CF911F91EC
:103DE0000895E5EFF1E085E0DF011D928A95E9F79E
:103DF0001092F4011092F301089587E196E00E9479
:103E00005D051F9281E08F931F9285E08F9389EC6F
:103E100095E09F938F930E94F6050F900F900F905F
:103E20000F900F900F9008958330E9F128F48130BE
:103E300061F0823009F10895853009F462C008F418
:103E400049C0863009F474C0089580911301262F6B
:103E500030E0280F311D2F3F310524F4680F6093A7
:103E6000130103C08FEF80931301809113011F9200
:103E70008F9382E095E072C080911201262F30E08E
:103E8000280F311D2F3F310524F4680F6093120174
:103E900003C08FEF80931201809112011F928F93C4
:103EA00080EF94E05BC080911101262F30E0280F55
:103EB000311D2F3F310524F4680F6093110103C0B9
:103EC0008FEF80931101809111011F928F938DEDDF
:103ED00094E044C080911001262F30E0280F311D5E
:103EE0002F3F310524F4680F6093100103C08FEF5A
:103EF00080931001809110011F928F9388EC94E0C1
:103F00002DC080910F01262F30E0280F311D2F3F4B
:103F1000310524F4680F60930F0103C08FEF809385
:103F20000F0180910F011F928F938FEA94E016C0CA
:103F300080910E01262F30E0280F311D2F3F3105D3
:103F400024F4680F60930E0103C08FEF80930E017D
:103F500080910E011F928F9384E994E09F938F9339
:103F60000E94F6050F900F900F900F9008958330E8
:103F700081F128F4813059F08230D1F008958530F4
:103F800009F449C0B8F1863009F456C0089580910B
:103F90001301681720F4861B8093130102C010924E
:103FA0001301809113011F928F9385E894E054C010
:103FB00080911201681720F4861B8093120102C0C1
:103FC00010921201809112011F928F9383E794E067
:103FD00043C080911101681720F4861B8093110162
:103FE00002C010921101809111011F928F9380E6FF
:103FF00094E032C080911001681720F4861B8093F2
:10400000100102C010921001809110011F928F9335
:104010008BE494E021C080910F01681720F4861B87
:1040200080930F0102C010920F0180910F011F9227
:104030008F9382E394E010C080910E01681720F402
:10404000861B80930E0102C010920E0180910E011A
:104050001F928F9387E194E09F938F930E94F605C0
:104060000F900F900F900F900895CF93C82F1F922D
:104070008F938CE197E09F938F930E94F60581E0E8
:1040800090E0A0E0B0E0BC01CD0104C0660F771F56
:10409000881F991FCA95D2F70E944A180F900F9057
:1040A0000F900F90CF910C944D14CF938732A8F5B9
:1040B0008E3108F02BC1803109F49FC0F8F48730AD
:1040C00009F464C0A8F4863009F024C18091EB01A2
:1040D000817F8E7F8093EB0181E297E00E945D05F6
:1040E0008BE09AE00E945D0581E08093FB014CC06B
:1040F0008B30F1F18E3009F46CC00CC1863109F4BB
:10410000B0C020F4813109F4EDC004C1893109F453
:1041100091C08B3109F449C0FDC0883349F150F496
:10412000893209F4F1C0853309F4EEC0873209F011
:10413000F1C0EAC0833409F4E7C028F48A3308F4F4
:10414000E9C08953E4C0883409F0E4C00E944D14EA
:104150008AEF99E00E945D052FEF83ED90E32150F7
:1041600080409040E1F700C000000E94F21B0CC0AC
:1041700088E497E05CC081EE99E00E945D05809143
:10418000EB0181608093EB01C1E0C9C08091EB013C
:10419000C82FC17080FFEFCF8DEE99E00E945D05C2
:1041A0008091EB01817F8E7F3DC09091EB0191FB6F
:1041B000CC27C0F981E0C827892FC0FB81F9809303
:1041C000EB01CC2319F084ED99E027C086EC99E04F
:1041D0002EC09091EB0192FBCC27C0F981E0C8275B
:1041E000892FC0FB82F98093EB01CC2319F087EB78
:1041F00099E013C087EA99E01AC09091EB0193FB14
:10420000CC27C0F981E0C827892FC0FB83F98093B0
:10421000EB01CC2351F08BE999E00E945D05809180
:10422000EB0181608093EB017AC08EE899E00E94F7
:104230005D05AACF8FE799E00E945D0582E599E0D0
:104240000E945D058BE199E00E945D058EEE98E08D
:104250000E945D0584EA98E00E945D0586E798E08B
:10426000E6CF88E698E00E945D050E94C10E1F928D
:104270008F938EE498E09F938F930E94F605809130
:104280000A011F928F9387E398E09F938F930E9478
:10429000F605809176011F928F9384E298E09F93B8
:1042A0008F930E94F60580910B011F928F9381E1FD
:1042B00098E09F938F930E94F6050E946B1B9F933B
:1042C0008F937F936F938AEF97E09F938F930E94D2
:1042D000F6058DB79EB746960FB6F8949EBF0FBEF3
:1042E0008DBF52CF0E944D14C0910B0181E0C827B1
:1042F000C0930B01CC2329F080EF97E00E945D056D
:104300000EC085EE97E093CF80E001C08D510E94F2
:1043100035203ACF83EE97E00E945D05C0E08C2FF8
:10432000CF91089580E0089580E00895CF93C82F3D
:104330008091FB01813071F020F0823009F44BC094
:1043400042C1E0910C01F0910D018081823209F0AF
:104350003CC107C0E0910C01F0910D0180818232D7
:1043600061F48C2F0E949221811104C08C2F0E9435
:1043700055202FC081E090E02CC08C2F0E9494210A
:10438000811126C0C431E1F070F4CB3081F0C0312E
:10439000D1F40E94FD1E84E197E00E945D0582E059
:1043A0008093FB0115C0C93259F0C83361F481E232
:1043B00097E00E945D0588E197E00E945D0508C0D6
:1043C0001092FB0104C182E197E00E945D05FFC0ED
:1043D00081E08170FEC0C43228F5CE3108F0C1C042
:1043E000CB30A1F1D0F4C73009F0D3C08EE1809377
:1043F000130182E3809312018AE08093110184E12A
:104400008093100188E080930F0188E280930E0171
:1044100088EB95E00E945D05BFC0C33149F1C4310E
:10442000C1F0B7C0CB3409F4A9C028F4C93289F06F
:10443000C83361F0AEC0C13509F49EC0C23509F47D
:1044400099C0CE3409F0A5C06AE09EC00E94FD1E4E
:10445000A3C08091FA01882319F01092FA019CC040
:1044600085EC95E00E945D0581E08093FB01B1C081
:104470008FE995E00E945D058DE895E00E945D055D
:10448000809113011F928F938AE895E09F938F93F9
:104490000E94F60588E895E00E945D0586E795E0B4
:1044A0000E945D05809112011F928F9383E795E032
:1044B0009F938F930E94F60581E795E00E945D052A
:1044C00082E695E00E945D05809111011F928F9315
:1044D0008FE595E09F938F930E94F6058DE595E01B
:1044E0000E945D058CE495E00E945D0580911001BD
:1044F0001F928F9389E495E09F938F930E94F60516
:1045000087E495E00E945D0582E395E00E945D05E9
:1045100080910F011F928F938FE295E09F938F936D
:104520000E94F6058DE295E00E945D0586E195E02A
:104530000E945D0580910E011F928F9383E195E0AB
:104540009F938F930E94F60581E195E00E945D059F
:104550008DB79EB748960FB6F8949EBF0FBE8DBF1D
:104560001BC0CE51EC2FF0E0E35DFE4F80818093C5
:10457000FA0112C061E003C061E006C06AE0809108
:10458000FA010E94141F08C08091FA010E94B71F0F
:1045900003C086EB95E013C08091FA01882369F08F
:1045A0001F928F9380EB95E09F938F930E94F60567
:1045B0000F900F900F900F9004C08DEA95E00E942D
:1045C0005D0581E006C01092FB0180E002C080E042
:1045D00000CFCF9108950E94F2226894B1110C94FB
:1045E000812308950E94662388F09F5798F0B92F81
:1045F0009927B751B0F0E1F0660F771F881F991F18
:104600001AF0BA95C9F714C0B13091F00E94802316
:10461000B1E008950C948023672F782F8827B85F26
:1046200039F0B93FCCF3869577956795B395D9F76F
:104630003EF490958095709561957F4F8F4F9F4F79
:104640000895E89409C097FB3EF490958095709585
:1046500061957F4F8F4F9F4F9923A9F0F92F96E9CE
:10466000BB279395F695879577956795B795F11143
:10467000F8CFFAF4BB0F11F460FF1BC06F5F7F4FE0
:104680008F4F9F4F16C0882311F096E911C07723F2
:1046900021F09EE8872F762F05C0662371F096E8FB
:1046A000862F70E060E02AF09A95660F771F881FCA
:1046B000DAF7880F9695879597F9089557FD9058E2
:1046C000440F551F59F05F3F71F04795880F97FBD6
:1046D000991F61F09F3F79F0879508951216130690
:1046E0001406551FF2CF4695F1DF08C016161706BF
:1046F0001806991FF1CF86957105610508940895F4
:10470000E894BB2766277727CB0197F908950E9485
:104710009A230C940B240E94FD2338F00E94042459
:1047200020F0952311F00C94F4230C94FA23112417
:104730000C9481230E945E2370F3959FC1F3950F23
:1047400050E0551F629FF001729FBB27F00DB11D15
:10475000639FAA27F00DB11DAA1F649F6627B00DA5
:10476000A11D661F829F2227B00DA11D621F739F8E
:10477000B00DA11D621F839FA00D611D221F749F9C
:104780003327A00D611D231F849F600D211D822FE3
:10479000762F6A2F11249F5750409AF0F1F088230A
:1047A0004AF0EE0FFF1FBB1F661F771F881F915037
:1047B0005040A9F79E3F510580F00C94F4230C94CF
:1047C00081235F3FE4F3983ED4F386957795679510
:1047D000B795F795E7959F5FC1F7FE2B880F911D61
:1047E0009695879597F9089597F99F6780E870E007
:1047F00060E008959FEF80EC089500240A94161657
:10480000170618060906089500240A9412161306BE
:10481000140605060895092E0394000C11F488234C
:1048200052F0BB0F40F4BF2B11F460FF04C06F5F68
:104830007F4F8F4F9F4F0895991B79E004C0991FB8
:10484000961708F0961B881F7A95C9F780950895EA
:1048500097FB072E16F4009407D077FD09D00E942D
:10486000422407FC05D03EF4909581959F4F089512
:10487000709561957F4F0895EE0FFF1F0590F4919D
:10488000E02D0994AA1BBB1B51E107C0AA1FBB1F47
:10489000A617B70710F0A61BB70B881F991F5A95CC
:1048A000A9F780959095BC01CD010895F894FFCFAC
:1048B0002A071B08F807C40790070101C901280847
:1048C000140A321E404D3622391A03CD0297027562
:1048D000023C02AF01C801E101FA011A0201020320
:0848E0000405060708090000A9
:106800000000000000000000040005000600070072
:10681000080009000A000B000C000D000E000F001C
:1068200010001100120013001400150016001700CC
:10683000180019001A001B001C001D001E001F007C
:10684000200021002200230024002500260027002C
:106850002800000035002B002C002D002E002F00FA
:1068600030002A00000033003400290036003700D1
:106870003800E00000000000000000000000000000
:106880000000000000000000000000000000000008
:1068900000000000000000000000000000000000F8
:1068A00000000000000000000000000000000000E8
:1068B00000000000000000000000000000000000D8
:1068C00000000000000000000000000000000000C8
:1068D00000000000000000000000000000000000B8
:1068E0000000000000000000310000000000000077
:1068F0000000E100E200E300F1A1E500E600E700AE
:106900000100010001000100EA4401000100E2442D
:106910000100010001005500460054004A004B00F0
:10692000560057004700480001000100E9440100FB
:106930000100010001000100010001003A003B00DC
:106940003C003D003E003F0040004100420043004B
:10695000580001004C00390001004400450052007D
:1069600001000100010050004F0081404D004E0029
:1069700051000100010001000100010001000100BF
:1069800001000100010001000100010001000100FF
:1069900001000100010001000100010001000100EF
:1069A00001000100010001000100010001000100DF
:1069B00001000100010001000100010001000100CF
:1069C00001000100010001000100010001000100BF
:1069D00001000100010001000100010001000100AF
:1069E0000100010001000100490001000100010057
:1069F000010001000100010001000100010001008F
:00000001FF
